:0200000480007A
:100000006F000005732F2034930F80006308FF03F7
:10001000930F90006304FF03930FB0006300FF038E
:10002000130F000063040F0067000F00732F2034CC
:1000300063540F006F00400093E19153171F0000BD
:1000400023223FFC171F000023200FFC6FF01FFF2F
:100050009300000013010000930100001302000050
:100060009302000013030000930300001304000038
:100070009304000013050000930500001306000020
:100080009306000013070000930700001308000008
:10009000930800001309000093090000130A0000F0
:1000A000930A0000130B0000930B0000130C0000D8
:1000B000930C0000130D0000930D0000130E0000C0
:1000C000930E0000130F0000930F0000732540F102
:1000D0006310050097020000938202017390523072
:1000E000735044749702000093820201739052305F
:1000F00073500018970200009382420273905230AE
:100100009B021000939252039382F2FF7390023B82
:100110009302F0017390023A73504030970200004E
:1001200093824201739052307350203073503030BC
:100130009301000097020000938202ED7390523009
:10014000130510001315F501635C05000F00F00F97
:10015000930110009308D005130500007300000000
:10016000970200009382820A638A02007390521001
:10017000B7B200009B82921073902230735000300F
:10018000371500001B05058073200530130520027C
:10019000732035309702000093824201739012342D
:1001A000732540F173002030930120001303800079
:1001B0009302001073B002109702000093820201B4
:1001C000739012147300201093011000730000004C
:1001D0006F008000631030020F00F00F6380010099
:1001E0009391110093E111009308D005138501004C
:1001F000730000000F00F00F930110009308D0056A
:100200001305000073000000F3222014F3235010A4
:1002100093F323006384030093F2F20FE39E62FAE8
:10022000970300009383C3FAF3221014E39672FA43
:100230006FF05FFC731000C00000000000000000C1
:1010000000000000000000000000000000000000E0
:1010100000000000000000000000000000000000D0
:1010200000000000000000000000000000000000C0
:1010300000000000000000000000000000000000B0
:081040000000000000000000A8
:040000058000000077
:00000001FF
